:1000000054C0BFC16DC06CC06BC06AC069C068C05D
:1000100067C066C065C064C063C062C061C060C0C4
:100020005FC05EC05DC01A034A00610067007500D2
:1000300061007200200041007400610072006900DC
:10004000180372006100700068006E0065007400A3
:100050002E006E0065007400040309040A033100D9
:1000600030003000300005010905A1010901A1009F
:1000700009300931150026FF00750895028102C07C
:100080000509190129111500250175019511810234
:10009000750195078103C012010101000000089B52
:1000A0002818000201010203010011241FBECFE540
:1000B000D4E0DEBFCDBF10E0A0E6B0E0E0E5FAE0BE
:1000C00002C005900D92A839B107D9F720E0A8E940
:1000D000B0E001C01D92A83EB207E1F70DD4B6C44E
:1000E0008FCFCF93C62F2091BD0024FF07C0209152
:1000F000BE0038E823272093BE0003C02AE52093E2
:10010000BD00DC01EFEBF0E09C2F9E0F8D91819301
:10011000892F8E1B1816D4F36C2F8FEB90E02DD106
:10012000CC5FC093BD00CF910895CF93DF938091B2
:10013000CE00835087FDA8C09091CB002091CA00CB
:100140002D3209F09FC0883009F09CC0CCE0D0E08F
:10015000C91BD109CE52DF4F83EC8093B2008AE5F0
:1001600080936100109298008881807619F0CE010A
:1001700070D27FC09A811092BB008981811106C024
:100180001092BC002BEB30E082E06FC0853019F498
:100190009093CF0067C0863009F04EC08B818130CC
:1001A00009F441C0823021F4CE0125D290E041C053
:1001B000833061F5911109C088E590E09093CD00FE
:1001C0008093CC0090E484E034C0913049F480E422
:1001D00090E09093CD008093CC0090E488E129C01A
:1001E000923049F486E290E09093CD008093CC0069
:1001F00090E48AE11EC09330D1F48CE590E09093B6
:10020000CD008093CC0090E48CE013C0813249F49F
:100210008BEA90E09093CD008093CC0090E489E04D
:1002200008C0823221F4CE01E6D190E402C090E40D
:1002300080E0909398001DC0883069F0893019F4EF
:100240009093D1000FC08A3049F08B3059F48BE481
:100250008093BE0007C021ED30E002C02BEB30E000
:1002600081E003C02BEB30E080E03093CD002093A1
:10027000CC009F81911104C09E81981708F4892FAA
:10028000809360001092CE008091610084FF46C090
:10029000809160008F3F09F441C0C82F893008F079
:1002A000C8E08C1B809360008091B20098E8892799
:1002B0008093B200CC2331F12091CC003091CD005D
:1002C0008091980086FF0BC0A3EBB0E0F9018C2F62
:1002D0008A0F94919D9331968A13FBCF09C0D9015F
:1002E000E3EBF0E08C2F8E0F9D9191938E13FCCF5A
:1002F0008FEF8C0F90E00196820F931F9093CD00AB
:100300008093CC006C2F83EB90E037D0CC5FCC3067
:1003100019F08FEF80936000C093610084E190B387
:10032000957031F48150D9F71092CF001092C90026
:10033000DF91CF91089585B7826085BF8BB78064C8
:100340008BBF8BE48093BE008AE58093BD00089547
:10035000A82FB92F80E090E041E050EA609530E0AE
:1003600009C02D9182279795879510F084279527AE
:10037000305EC8F36F5FA8F30895EADF8D939D9315
:100380000895CF93CFB7CF93C395809BE9F7809B18
:1003900009C0809B07C0809B05C0809B03C0809BD9
:1003A00001C0A3C0DF93C091CB00DD27CE52DF4F49
:1003B000809B02C0DF91EBCF2F930F931F9300B36D
:1003C0002FEF00FB20F94F933F9310B34FEF01271E
:1003D00000FB21F93BE031C04E7F012F10B32160BB
:1003E00028C0102F4D7F2260000000B329C04B7F32
:1003F0002460012F000010B32BC010B3477F28608A
:100400002AC04F7E00B320612CC04F7D10B3206204
:100410002FC04F7B00B3206432C0422700B3499302
:100420004FEF0000102710FB20F910B31570C9F131
:10043000297F91F2012700FB21F900B3237F89F284
:10044000315058F1102710FB22F910B3277E79F2B2
:10045000012700FB23F92F7C81F200B3102710FB4A
:1004600024F92F7971F200C010B3012700FB25F9A0
:100470002F7359F200C000B3102710FB26F9223069
:1004800040F200C010B3012700FB27F9243028F602
:100490004F77206810B30000F9CF10E41ABF00278F
:1004A00019C03B503195C31BD04010E41ABF0881DE
:1004B000033CF9F00B34E9F02091C9001981110FC8
:1004C0001213EDCF4A81441F093641F10D3211F06C
:1004D000013E29F70093D0003F914F911F910F915A
:1004E0002F91DF91CAB7C6FD4FCFCF91CFBFCF912C
:1004F00018952091D000222379F31091CE0011237A
:1005000069F534306AF13093CE002093CA0010911F
:10051000CB003BE0311B3093CB0022C00091CE00DA
:100520000130E4F40AE54F7049F43091610034FD84
:1005300019C000936100C2EBD0E018C03091BD003B
:1005400034FD10C00093BD00CEEBD0E00FC0279566
:10055000A8F45150A9F4220F0000F9CF4AE503C0D6
:1005600042ED01C0432FC4E1D0E032E011B3156089
:10057000909A11BB02B320E415E05F93012756E087
:1005800002BB279520F4515021F4220FF9CF012707
:1005900056E000003B5A02BBD0F2279528F4515098
:1005A00029F4220F0000F9CF012756E0279502BB5E
:1005B00020F4515021F4220FF9CF012756E0299160
:1005C000332302BB21F60A7F1091CF00110FC651D1
:1005D000D04002BB11F01093C90010E41ABF0160B3
:1005E00011B31A7F402F4A7F5F9100C000C002BB49
:1005F00011BB42BB71CFFC018081807641F59181B6
:10060000963031F593819230D1F0923269F0913089
:10061000F9F48091A3009091A4009093CD00809371
:10062000CC008091A20008958091A6009091A7002F
:100630009093CD008093CC008091A500089582E630
:1006400090E09093CD008093CC0082E2089580E00A
:1006500008952AE930E03093CD002093CC00FC01CE
:1006600020812076203299F48181813081F4E091DB
:10067000A000F091A1000088F189E02D8AE990E0C6
:100680000995E091A000F091A1008081089580E09B
:100690000895009741F025E0EDEAF0E0DC010190DB
:1006A0000D922A95E1F785E0EDEAF0E0A8EAB0E0E6
:1006B00001900D928A95E1F70895EF92FF921F93B2
:1006C000CF93DF93CDB7DEB767970FB6F894DEBF51
:1006D0000FBECDBF80E88A8389831B821C821D8266
:1006E0001E821F827E0188E0E80EF11C8CE0D7019B
:1006F0001D928A95E9F7FE01749680E090E040E251
:1007000050E09A01082E02C0359527950A94E2F729
:1007100065B3122F1095612365BB64B3622B64BB74
:10072000AFE6B7E11197F1F700C0000073B3737043
:10073000708366B368736695672B6083B09B02C055
:100740006062608334B3312334BB35B3322B35BBA5
:100750000196319684309105A1F69F8981E091FB45
:10076000662760F968276F835C89752F7170782719
:100770007E834D89E42FE170E827ED833E89F32FD6
:10078000F170F827FC83292F217028272B8354FB35
:10079000112710F918271A8744FB112710F9182779
:1007A000198734FB112710F91827188794FD02C008
:1007B0008FEF898311E053FB882780F981278D878C
:1007C00043FB882780F981278C8733FB882780F9B2
:1007D00081278B8793FF198211E052FB882780F9CC
:1007E0008127888B42FB882780F981278F8732FBFE
:1007F000882780F981278E8792FD02C08FEF8A8338
:1008000081E055FB552750F958275B8B45FB442762
:1008100040F948274A8B35FB332730F93827398B85
:1008200095FF1A82F1112260E11124607111286094
:1008300061112061F70180E090E030E241914111C7
:10084000232B0196330F83309105C1F780E090E0B0
:1008500041E030E0E4E0F0E0EC0FFD1FE80FF91FAD
:1008600067816111342B440F01968830910591F70F
:1008700089818093AD008A818093AE002093AF0080
:100880003093B0005093B10067960FB6F894DEBF76
:100890000FBECDBFDF91CF911F91FF90EF900895D4
:1008A000CF93CFB7F89414BA8FEF85BB17BA88BB34
:1008B00004DFCFBFCF91089580918400909185008F
:1008C000892B31F0109285001092840081E0089508
:1008D00045E050E068EA70E08DEA90E0AAD0089523
:1008E00086E690E090938B0080938A0086E890E003
:1008F000089582E190E0089581E087BB8EEF88BB88
:1009000014BA8FEF85BB88EF82BB85E081BB83BFC4
:100910008FE085BD82E383BDE3DFFC019093A100FE
:100920008093A000848195819093A7008093A60076
:1009300082818093A50080859185009731F0909306
:10094000A4008093A300868107C087E990E090937C
:10095000A4008093A300CDDF8093A2008091A50026
:1009600080937B002FE088E190E00FB6F894A89583
:1009700081BD0FBE21BDE091A000F091A1000284D5
:10098000F385E02D0995D7DC82B38A7F82BB81B3E2
:10099000856081BB87EC9FEA0197F1F700C00000FA
:1009A00081B38A7F81BB789411E0D0E0C0E8A8953C
:1009B000BCDB112341F0E091A000F091A100048480
:1009C000F585E02D099508B607FE16C0C8BFD11100
:1009D00015C0E091A000F091A1000484F585E02D00
:1009E0000995E091A000F091A1000684F785E02D23
:1009F0000995811103C01BC0DD23C9F08091BD00A2
:100A000084FD03C0D1E010E0D2CFE091A000F091CE
:100A1000A1000088F189E02D8AE990E00995E09134
:100A2000A000F091A10060818AE990E05ADBD0E05B
:100A3000EACFFB01DC0104C08D910190801921F403
:100A400041505040C8F7881B990B0895F894FFCF88
:100A5000FF5A0902220001010000320904000001CE
:100A600003000000092101010001220000070581A7
:100A70000308000A0100050031000000000000002A
:080A800050045D035C0449030E
:00000001FF
